:100000000C9462060C948A060C948A060C948A0658
:100010000C948A060C948A060C948A060C948A0620
:100020000C948A060C948A060C948A060C948A0610
:100030000C948A060C948A060C948A060C948A0600
:100040000C94B7070C948A060C948A060C948A06C2
:100050000C948A060C948A060C948A060C948A06E0
:100060000C948A060C948A06FFFEFDFCFBFAF9F854
:10007000F7F6F5F4F3F2F1F0EFEEEDECEBEBEAE985
:10008000E8E7E6E5E4E3E2E1E0E0DFDEDDDCDBDA61
:10009000D9D9D8D7D6D5D4D3D3D2D1D0CFCECECD2F
:1000A000CCCBCACAC9C8C7C6C6C5C4C3C2C2C1C0F0
:1000B000BFBFBEBDBCBCBBBAB9B9B8B7B6B6B5B4A4
:1000C000B3B3B2B1B1B0AFAEAEADACACABAAAAA94E
:1000D000A8A8A7A6A6A5A4A4A3A2A2A1A0A09F9EEB
:1000E0009E9D9D9C9B9B9A9999989897969695957D
:1000F00094939392929190908F8F8E8E8D8C8C8B07
:100100008B8A8A8988888787868685858484838385
:1001100082818180807F7F7E7E7D7D7C7C7B7B7AFF
:100120007A7979787877777676757575747473736C
:100130007272717170706F6F6F6E6E6D6D6C6C6BD3
:100140006B6B6A6A69696868686767666665656532
:100150006464636363626261616160605F5F5F5E8C
:100160005E5D5D5D5C5C5C5B5B5A5A5A59595958DF
:10017000585857575656565555555454545353532B
:100180005252525151515050504F4F4F4E4E4E4D72
:100190004D4D4C4C4C4B4B4B4A4A4A4A49494948B5
:1001A00048484747474746464645454545444444F1
:1001B0004343434342424241414141404040403F2A
:1001C0003F3F3E3E3E3E3D3D3D3D3C3C3C3C3B3B5F
:1001D0003B3B3A3A3A3A393939393838383838378E
:1001E00037373736363636353535353534343434B9
:1001F00033333333333232323231313131313030E3
:100200003030302F2F2F2F2F2E2E2E2E2E2D2D2D06
:100210002D2D2C2C2C2C2C2B2B2B2B2B2B2A2A2A28
:100220002A2A292929292929282828282828272746
:100230002727272626262626262525252525252562
:10024000242424242424232323232323222222227C
:100250002222222121212121212120202020202091
:10026000201F1F1F1F1F1F1F1E1E1E1E1E1E1E1DA6
:100270001D1D1D1D1D1D1D1C1C1C1C1C1C1C1C1BB8
:100280001B1B1B1B1B1B1B1A1A1A1A1A1A1A1A19C8
:1002900019191919191919191818181818181818D6
:1002A00017171717171717171717161616161616E4
:1002B00016161615151515151515151515141414EE
:1002C00014141414141414131313131313131313F7
:1002D00013131212121212121212121212121111FE
:1002E0001111111111111111111010101010101005
:1002F0001010101010100F0F0F0F0F0F0F0F0F0F08
:100300000F0F0F0E0E0E0E0E0E0E0E0E0E0E0E0E0A
:100310000D0D0D0D0D0D0D0D0D0D0D0D0D0D0D0C0E
:100320000C0C0C0C0C0C0C0C0C0C0C0C0C0C0B0B0F
:100330000B0B0B0B0B0B0B0B0B0B0B0B0B0B0A0A0F
:100340000A0A0A0A0A0A0A0A0A0A0A0A0A0A0A0A0D
:10035000090909090909090909090909090909090D
:10036000090908080808080808080808080808080B
:100370000808080808080707070707070707070707
:100380000707070707070707070707070606060601
:1003900006060606060606060606060606060606FD
:1003A00006060606050505050505050505050505F9
:1003B00005050505050505050505050505050404EF
:1003C00004040404040404040404040404040404ED
:1003D00004040404040404040404040303030303E2
:1003E00003030303030303030303030303030303DD
:1003F00003030303030303030303030302020202D1
:1004000002020202020202020202020202020202CC
:1004100002020202020202020202020202020202BC
:1004200002020101010101010101010101010101BA
:1004300001010101010101010101010101010101AC
:10044000010101010101010101010101010101009D
:10045000000000000000000000000000000000009C
:100460000000000000000000000005000A000F006E
:10047000140019001E00230027002C003100360054
:100480003B003F00440049004D00520057005B0014
:100490006000640069006D00720076007B007F00E0
:1004A000840088008C009100950099009E00A200B5
:1004B000A600AA00AE00B300B700BB00BF00C30097
:1004C000C700CB00CF00D300D700DB00DF00E30084
:1004D000E700EB00EF00F300F600FA00FE00020177
:1004E000060109010D011101140118011C011F0170
:1004F000230127012A012E013101350138013C0178
:100500003F01430146014A014D0150015401570189
:100510005B015E016101640168016B016E017101A3
:10052000750178017B017E018101850188018B01C4
:100530008E019101940197019A019D01A001A301EF
:10054000A601A901AC01AF01B201B501B801BB011F
:10055000BD01C001C301C601C901CB01CE01D1015A
:10056000D401D701D901DC01DF01E101E401E70198
:10057000E901EC01EF01F101F401F601F901FB01E0
:10058000FE0101020302060208020B020D020F0225
:1005900012021402170219021C021E022002230278
:1005A000250227022A022C022E02310233023502D2
:1005B00038023A023C023E02400243024502470230
:1005C00049024B024E025002520254025602580295
:1005D0005A025C025E0260026302650267026902FF
:1005E0006B026D026F02710273027502770278026C
:1005F0007A027C027E0280028202840286028802E3
:100600008A028B028D028F0291029302950296025A
:1006100098029A029C029D029F02A102A302A402D8
:10062000A602A802AA02AB02AD02AF02B002B20259
:10063000B402B502B702B902BA02BC02BD02BF02DF
:10064000C102C202C402C502C702C802CA02CC0269
:10065000CD02CF02D002D202D302D502D602D802F6
:10066000D902DB02DC02DD02DF02E002E202E30289
:10067000E502E602E702E902EA02EC02ED02EE021E
:10068000F002F102F202F402F502F602F802F902B7
:10069000FA02FC02FD02FE02FF0201030203030351
:1006A00005030603070308030A030B030C030D03EA
:1006B0000E0310031103120313031403160317038D
:1006C000180319031A031B031D031E031F03200332
:1006D00021032203230324032503270328032903DB
:1006E0002A032B032C032D032E032F033003310386
:1006F0003203330334033503360337033803390336
:100700003A033B033C033D033E033F0340034103E5
:100710004203430344034503460347034803490395
:100720004A034B034B034C034D034E034F0350034B
:100730005103520353035303540355035603570302
:100740005803590359035A035B035C035D035E03BB
:100750005E035F0360036103620363036303640377
:100760006503660366036703680369036A036A0334
:100770006B036C036D036D036E036F0370037003F3
:1007800071037203720373037403750375037603B5
:10079000770377037803790379037A037B037C0378
:1007A0007C037D037E037E037F037F03800381033D
:1007B0008103820383038303840385038503860304
:1007C000870387038803880389038A038A038B03CB
:1007D0008B038C038D038D038E038E038F03900395
:1007E0009003910391039203920393039403940360
:1007F000950395039603960397039703980398032D
:10080000990399039A039B039B039C039C039D03F9
:100810009D039E039E039F039F03A003A003A103C8
:10082000A103A203A203A303A303A403A403A50398
:10083000A503A503A603A603A703A703A803A8036C
:10084000A903A903AA03AA03AB03AB03AB03AC033D
:10085000AC03AD03AD03AE03AE03AE03AF03AF0312
:10086000B003B003B103B103B103B203B203B303E6
:10087000B303B303B403B403B503B503B503B603BD
:10088000B603B703B703B703B803B803B903B90393
:10089000B903BA03BA03BA03BB03BB03BB03BC036C
:1008A000BC03BD03BD03BD03BE03BE03BE03BF0344
:1008B000BF03BF03C003C003C003C103C103C1031F
:1008C000C203C203C203C303C303C303C403C403F9
:1008D000C403C503C503C503C603C603C603C703D4
:1008E000C703C703C703C803C803C803C903C903B1
:1008F000C903CA03CA03CA03CA03CB03CB03CB038E
:10090000CC03CC03CC03CC03CD03CD03CD03CE036A
:10091000CE03CE03CE03CF03CF03CF03CF03D00349
:10092000D003D003D103D103D103D103D203D20327
:10093000D203D203D303D303D303D303D403D40307
:10094000D403D403D503D503D503D503D503D603E8
:10095000D603D603D603D703D703D703D703D803C9
:10096000D803D803D803D803D903D903D903D903AB
:10097000DA03DA03DA03DA03DA03DB03DB03DB038C
:10098000DB03DB03DC03DC03DC03DC03DC03DD0370
:10099000DD03DD03DD03DD03DE03DE03DE03DE0353
:1009A000DE03DF03DF03DF03DF03DF03E003E00336
:1009B000E003E003E003E103E103E103E103E1031A
:1009C000E103E203E203E203E203E203E203E303FF
:1009D000E303E303E303E303E403E403E403E403E3
:1009E000E403E403E503E503E503E503E503E503C9
:1009F000E503E603E603E603E603E603E603E703AF
:100A0000E703E703E703E703E703E703E803E80394
:100A1000E803E803E803E803E803E903E903E9037B
:100A2000E903E903E903E903EA03EA03EA03EA0362
:100A3000EA03EA03EA03EB03EB03EB03EB03EB0349
:100A4000EB03EB03EB03EC03EC03EC03EC03EC0331
:100A5000EC03EC03ED03ED03ED03ED03ED03ED0318
:100A6000ED03ED03ED03EE03EE03EE03EE03EE0301
:100A7000EE03EE03EE03EF03EF03EF03EF03EF03E9
:100A8000EF03EF03EF03EF03F003F003F003F003D2
:100A9000F003F003F003F003F003F103F103F103BB
:100AA000F103F103F103F103F103F103F103F203A5
:100AB000F203F203F203F203F203F203F203F2038E
:100AC000F203F203F303F303F303F303F303F30378
:100AD000F303F303F303F303F403F403F403F40362
:100AE000F403F403F403F403F403F403F403F4034E
:100AF000F503F503F503F503F503F503F503F50336
:100B0000F503F503F503F503F603F603F603F60321
:100B1000F603F603F603F603F603F603F603F6030D
:100B2000F603F703F703F703F703F703F703F703F6
:100B3000F703F703F703F703F703F703F803F803E3
:100B4000F803F803F803F803F803F803F803F803CD
:100B5000F803F803F803F803F803F903F903F903BA
:100B6000F903F903F903F903F903F903F903F903A5
:100B7000F903F903F903F903F903FA03FA03FA0392
:100B8000FA03FA03FA03FA03FA03FA03FA03FA037D
:100B9000FA03FA03FA03FA03FA03FA03FB03FB036B
:100BA000FB03FB03FB03FB03FB03FB03FB03FB0355
:100BB000FB03FB03FB03FB03FB03FB03FB03FB0345
:100BC000FB03FC03FC03FC03FC03FC03FC03FC032E
:100BD000FC03FC03FC03FC03FC03FC03FC03FC031D
:100BE000FC03FC03FC03FC03FC03FD03FD03FD030A
:100BF000FD03FD03FD03FD03FD03FD03FD03FD03F5
:100C0000FD03FD03FD03FD03FD03FD03FD03FD03E4
:100C1000FD03FD03FD03FD03FE03FE03FE03FE03D0
:100C2000FE03FE03FE03FE03FE03FE03FE03FE03BC
:100C3000FE03FE03FE03FE03FE03FE03FE03FE03AC
:100C4000FE03FE03FE03FE03FE03FE03FF03FF039A
:100C5000FF03FF03FF03FF03FF03FF03FF03FF0384
:100C6000FF03FF03FF03FF03000000002400270031
:100C70002A0000000000250028002B0000000000D2
:100C800023002600290004040404040404040202CE
:100C900002020202030303030303010204081020FB
:100CA0004080010204081020010204081020000006
:100CB000000800020100000304070000000000001B
:100CC0000000680A11241FBECFEFD8E0DEBFCDBF01
:100CD00011E0A0E0B1E0E4EBF9E102C005900D9273
:100CE000A030B107D9F721E0A0E0B1E001C01D922A
:100CF000A432B207E1F716E0C2E6D6E004C02197BD
:100D0000FE010E94D20CC136D107C9F70E9401082A
:100D10000C94D80C0C940000833081F028F48130BE
:100D200099F08230A9F008958730A9F08830C9F091
:100D30008430B1F4809180008F7D03C08091800069
:100D40008F7780938000089584B58F7784BD089550
:100D500084B58F7DFBCF8091B0008F778093B000FA
:100D600008958091B0008F7DF9CFCF93DF93282F26
:100D700030E0F901E255F34F8491F901E656F34F63
:100D8000D491F901EA57F34FC491CC23A1F081111A
:100D90000E948C06EC2FF0E0EE0FFF1FE458F34F9B
:100DA000A591B491EC91ED2381E090E009F480E00D
:100DB000DF91CF91089580E090E0FACF1F93CF9319
:100DC000DF93282F30E0F901E255F34F8491F901C8
:100DD000E656F34FD491F901EA57F34FC491CC236F
:100DE000A9F0162F81110E948C06EC2FF0E0EE0F77
:100DF000FF1FEE58F34FA591B4918FB7F894EC9183
:100E0000111108C0D095DE23DC938FBFDF91CF9105
:100E10001F910895DE2BF8CFCF93DF9390E0FC0174
:100E2000E656F34F24918A57934FFC01849188230F
:100E3000C9F090E0880F991FFC01E859F34FA59184
:100E4000B491FC01EE58F34FC591D49161110DC0DE
:100E50009FB7F8948C91209582238C9388812823C6
:100E600028839FBFDF91CF910895623051F49FB7DF
:100E7000F8943C91822F809583238C93E8812E2BCC
:100E8000EFCF8FB7F894EC912E2B2C938FBFEACF36
:100E90001F93CF93DF93182FEB0161E00E940C07A3
:100EA000209739F460E0812FDF91CF911F910C944E
:100EB000DE06CF3FD10511F461E0F5CFE12FF0E080
:100EC000E255F34FE491E33031F140F4E130B1F019
:100ED000E230E1F0C038D1057CF7E4CFE73029F10A
:100EE000E83059F1E430B1F780918000806280935E
:100EF0008000D0938B00C0938A0004C084B58068C2
:100F000084BDC7BDDF91CF911F91089584B58062E4
:100F100084BDC8BDF7CF8091800080688093800039
:100F2000D0938900C0938800EDCF8091B000806895
:100F30008093B000C093B300E5CF8091B000806291
:100F40008093B000C093B400DDCF8E508064809356
:100F50007C0080917A00806480937A0080917A008E
:100F600086FDFCCF809178009091790008951F92C2
:100F70000F920FB60F9211242F933F938F939F934D
:100F8000AF93BF938091200190912101A091220104
:100F9000B091230130911F0123E0230F2D3758F525
:100FA0000196A11DB11D20931F01809320019093F4
:100FB0002101A0932201B093230180911B01909104
:100FC0001C01A0911D01B0911E010196A11DB11D32
:100FD00080931B0190931C01A0931D01B0931E01EF
:100FE000BF91AF919F918F913F912F910F900FBE25
:100FF0000F901F90189526E8230F0296A11DB11D92
:10100000D2CFCF93DF9300D000D0CDB7DEB77894A6
:1010100084B5826084BD84B5816084BD85B58260FD
:1010200085BD85B5816085BD80916E0081608093AE
:101030006E00109281008091810082608093810017
:101040008091810081608093810080918000816027
:10105000809380008091B10084608093B100809182
:10106000B00081608093B00080917A0084608093AA
:101070007A0080917A00826080937A0080917A0071
:10108000816080937A0080917A00806880937A00F2
:101090001092C10062E084E00E940C0760E081E1F0
:1010A0000E940C0761E083E00E940C0761E089E088
:1010B0000E940C0761E08AE00E940C0761E08BE06F
:1010C0000E940C0783E28093B00081E08093B1001E
:1010D00082E88093800089E1809381008FEF90E027
:1010E000909387008093860000E014E066246A9461
:1010F000712C812C912C54018A948FB7F894C09054
:101100002001D0902101E0902201F09023018FBFB7
:10111000C0921701D0921801E0921901F0921A01C1
:1011200084E00E94B50620911401211103C091E0D2
:10113000813009F090E090931501213011F491E095
:10114000811190E090931601809314019923E9F0A6
:101150008091120190911301029709F023C18091AF
:1011600010019091110190930F0180930E0121E0E5
:1011700030E0309313012093120110920A01109273
:101180000B0110920C0110920D0181E10E94B50635
:1011900020910701211103C091E0813009F090E016
:1011A00090930801213009F4811120E02093090176
:1011B000809307019923E9F0809112019091130126
:1011C000029709F0F4C08091100190911101909361
:1011D0000F0180930E0141E050E0509313014093C2
:1011E000120110920A0110920B0110920C01109240
:1011F0000D018EE00E94A507FC01EE0FFF1FE859CC
:10120000FB4F859194919C838B838FE00E94A5076F
:10121000FC01EE0FFF1FE859FB4F259134913A83F3
:10122000298380E10E94A5074091030150910401A8
:1012300060910501709106014C155D056E057F05F5
:1012400009F4A8C0A801EB81FC814E1B5F0B5C83F5
:101250004B83C0920301D0920401E0920501F09209
:1012600006014D3F5340CCF0209112013091130103
:101270002130310591F422E030E0309313012093C6
:10128000120140E050E060E874E440930A0150939A
:101290000B0160930C0170930D01209112013091AC
:1012A00013012115310509F087C010921101109228
:1012B000100140911001509111015A834983BA01E4
:1012C0008BE00E94480720EAE981FA812E9FC00145
:1012D0002F9F900D1124B3010E94A30C83E00E9464
:1012E0004807B30149815A81641B750B8AE00E944B
:1012F00048076091020189E00E94DE06C0900A0161
:10130000D0900B01E0900C01F0900D0120E030E056
:1013100040E854E4C701B6010E94310C181684F469
:1013200020E030E040E055E4C701B6010E94440BE4
:1013300087FF06C082E090E0909313018093120132
:1013400020E030E040E055E4C701B6010E94310CD6
:1013500087FD0FC010920A0110920B0110920C0130
:1013600010920D01109213011092120191E09093CE
:10137000020180910201882369F08091000190911F
:10138000010101968B3091050CF09BC090930101F7
:1013900080930001E0E0F0E0EF2B09F4AECE0E9474
:1013A0000000ABCE10920F0110920E01E0CE109211
:1013B0000F0110920E010FCF7C0197FF03C043E095
:1013C000E40EF11CF594E794F594E79420900A015B
:1013D00030900B0140900C0150900D0121303105EF
:1013E00009F04CC0C201B1010E94490B68597F4FFE
:1013F000FB01649120910E0130910F01032E000C2E
:10140000440B550B2F5F310941095109A62FB0E05C
:101410000E94930AA50194010E94740A21503F4F33
:101420004F4F5F4FD7010E949E0AA50194010E9471
:10143000740A30931101209310012B813C81B90172
:10144000330F880B990B0E94810B2DEC3CEC4CE484
:101450005DE30E94360C20E030E040E05FE30E9454
:10146000360CA20191010E94D80A60930A01709380
:101470000B0180930C0190930D011BCF223031059D
:1014800009F017CFC201B1010E94490B745068598D
:101490007F4FFB01249130E0D7010E94B70CA501DA
:1014A00094010E94740A3093110120931001B80135
:1014B00029813A81621B730B072E000C880B990B54
:1014C000C2CF10920101109200011092020162CF6E
:1014D000E4E1F1E081E0808311821282E7E0F1E053
:1014E0001082118212820895052E97FB1EF400943B
:1014F0000E948B0A57FD07D00E94A60A07FC03D062
:101500004EF40C948B0A50954095309521953F4FA1
:101510004F4F5F4F089590958095709561957F4FDF
:101520008F4F9F4F08950E94C80AA59F900DB49FAA
:10153000900DA49F800D911D11240895B7FF0C9468
:10154000930A0E94930A821B930B0895A1E21A2E1C
:10155000AA1BBB1BFD010DC0AA1FBB1FEE1FFF1F57
:10156000A217B307E407F50720F0A21BB30BE40BA7
:10157000F50B661F771F881F991F1A9469F76095EE
:101580007095809590959B01AC01BD01CF010895A8
:10159000A29FB001B39FC001A39F700D811D1124B4
:1015A000911DB29F700D811D1124911D08955058F9
:1015B000BB27AA270E94EF0A0C94F70B0E94E90BA5
:1015C00038F00E94F00B20F039F49F3F19F426F414
:1015D0000C94E60B0EF4E095E7FB0C94E00BE92F7E
:1015E0000E94080C58F3BA1762077307840795071F
:1015F00020F079F4A6F50C942A0C0EF4E0950B2E4D
:10160000BA2FA02D0B01B90190010C01CA01A00154
:101610001124FF27591B99F0593F50F4503E68F1AF
:101620001A16F040A22F232F342F4427585FF3CFF0
:10163000469537952795A795F0405395C9F77EF4C1
:101640001F16BA0B620B730B840BBAF09150A1F00A
:10165000FF0FBB1F661F771F881FC2F70EC0BA0F90
:10166000621F731F841F48F4879577956795B79518
:10167000F7959E3F08F0B0CF9395880F08F0992713
:10168000EE0F9795879508950E94BC0B08F481E0B2
:1016900008950E94500B6894B1110C942B0C08957E
:1016A0000E94100C88F09F5798F0B92F9927B751D6
:1016B000B0F0E1F0660F771F881F991F1AF0BA95F6
:1016C000C9F714C0B13091F00E942A0CB1E008951E
:1016D0000C942A0C672F782F8827B85F39F0B93F10
:1016E000CCF3869577956795B395D9F73EF49095A9
:1016F0008095709561957F4F8F4F9F4F0895E89427
:1017000009C097FB3EF490958095709561957F4F49
:101710008F4F9F4F9923A9F0F92F96E9BB279395F7
:10172000F695879577956795B795F111F8CFFAF407
:10173000BB0F11F460FF1BC06F5F7F4F8F4F9F4F38
:1017400016C0882311F096E911C0772321F09EE896
:10175000872F762F05C0662371F096E8862F70E0FC
:1017600060E02AF09A95660F771F881FDAF7880FD6
:101770009695879597F90895990F0008550FAA0B2C
:10178000E0E8FEEF16161706E807F907C0F0121694
:101790001306E407F50798F0621B730B840B950B97
:1017A00039F40A2661F0232B242B252B21F40895EC
:1017B0000A2609F4A140A6958FEF811D811D089589
:1017C00097F99F6780E870E060E008959FEF80ECF4
:1017D000089500240A941616170618060906089597
:1017E00000240A9412161306140605060895092EFD
:1017F0000394000C11F4882352F0BB0F40F4BF2B6C
:1018000011F460FF04C06F5F7F4F8F4F9F4F0895AB
:1018100057FD9058440F551F59F05F3F71F04795A1
:10182000880F97FB991F61F09F3F79F08795089586
:10183000121613061406551FF2CF4695F1DF08C0A5
:10184000161617061806991FF1CF869571056105C2
:1018500008940895E894BB2766277727CB0197F96A
:1018600008950E94BC0B08F48FEF08950E94490C64
:101870000C94F70B0E94E90B38F00E94F00B20F05B
:10188000952311F00C94E00B0C94E60B11240C94AE
:101890002B0C0E94080C70F3959FC1F3950F50E03C
:1018A000551F629FF001729FBB27F00DB11D639F12
:1018B000AA27F00DB11DAA1F649F6627B00DA11DB8
:1018C000661F829F2227B00DA11D621F739FB00D5E
:1018D000A11D621F839FA00D611D221F749F3327CE
:1018E000A00D611D231F849F600D211D822F762F67
:1018F0006A2F11249F5750409AF0F1F088234AF044
:10190000EE0FFF1FBB1F661F771F881F91505040AF
:10191000A9F79E3F510580F00C94E00B0C942B0C22
:101920005F3FE4F3983ED4F3869577956795B79536
:10193000F795E7959F5FC1F7FE2B880F911D969550
:10194000879597F9089597FB072E16F4009407D012
:1019500077FD09D00E94BE0C07FC05D03EF490959F
:1019600081959F4F0895709561957F4F08950E94CE
:10197000C80AB7FF0895821B930B0895AA1BBB1BCF
:1019800051E107C0AA1FBB1FA617B70710F0A61B7F
:10199000B70B881F991F5A95A9F780959095BC01A0
:1019A000CD010895EE0FFF1F0590F491E02D0994ED
:0419B000F894FFCFD9
:00000001FF
